:1000000002016A02019000000000003200000000BE
:10001000000000320000000000000032000000007C
:100020000000003200000000000000000000C39546
:10003000F02212002E60044002E422740122780FA4
:10004000790BE766A2E75006E7A2E774FF22E50B0B
:10005000B50F12E50AB50E0DE509B50D08E508B5B1
:100060000C03C3E42274FF2202003EAE02E6F7084E
:1000700009DEFA227B0474FA311FDBFADAF622C0B9
:10008000E07403311FD0E0220022D2B51188D2B033
:1000900011887F0AD330B50C30B009DFF8C2B01137
:1000A00088C2B5C3920422C2B01188D2B51188D2D9
:1000B000B02292B01188500C7F0A20B007DFFBD22B
:1000C000B5D38013D2B511887F0A20B507DFFBD2E4
:1000D000B0D38003C2B5C322D2B01188D2B5118883
:1000E0007F0A20B505DFFBD38007A2B092D5C2B549
:1000F000C3227E083311B2400CDEF911D84006A2AB
:10010000D5500211A792042233FD7E0811D8400C6D
:10011000A2D533DEF7CD13CD11B2D2B0920422783E
:10012000A37901D8FED9FCD5E0F522C3AE02E637AB
:10013000F70809DEF9227408C0F08502F0A4FFD0A8
:10014000F078103159C37810316178083161500668
:10015000780C7910312BDFED22AE02760008DEFB41
:1001600022AE02E633F608DEFA22787FE4F6D8FD06
:100170007581477520007590FF75B0FFC2B4D2AF8E
:10018000D2A8C294C295C296C29743870202018246
:10019000C0D0C2D3C0E0C0F0C083C082C000C001E4
:1001A000C002C003C004C005C006C007C008C00923
:1001B000C00AC00BC00CC00DC00EC00FC010C011D3
:1001C000C012C013E53BB43202800250030201D3D7
:1001D000438702D294D295D296D29775370075365E
:1001E00000753900752300752400752500752600FB
:1001F0007533000539D294C29775220C300505304D
:100200009312C20520930D742812011F209305D26A
:10021000051203A575220A300605309212C2062087
:10022000920D742812011F209205D2061203A575A3
:10023000220B300705309112C20720910D7428124D
:10024000011F209105D2071203A5D297C2967522ED
:1002500009300505309312C20520930D7428120150
:100260001F209305D2051203A5752208300605301C
:100270009212C20620920D742812011F209205D2FC
:10028000061203A5752207300705309112C2072018
:10029000910D742812011F209105D2071203A5D2D7
:1002A00096C295752206300505309312C20520933B
:1002B0000D742812011F209305D2051203A5752283
:1002C00005300605309212C20620920D74281201E4
:1002D0001F209205D2061203A575220430070530AF
:1002E0009112C20720910D742812011F209105D28E
:1002F000071203A5D295C2947522033005053093E9
:1003000012C20520930D742812011F209305D205F7
:100310001203A5752202300605309212C206209201
:100320000D742812011F209205D2061203A5752212
:1003300001300705309112C20720910D7428120177
:100340001F209105D2071203A5300805209012C284
:100350000830900D742812011F309005D208120643
:1003600012740A311FE539B4FA0280025003020107
:10037000F3D013D012D011D010D00FD00ED00DD09A
:100380000CD00BD00AD009D008D007D006D005D0A9
:1003900004D003D002D001D000D082D083D0F0D0DE
:1003A000E0D0D03222753900D2B37464311FC2B3A9
:1003B0007432311FA293920450030203C2740102EB
:1003C00003C3E4C0E0A292920450030203D3740179
:1003D0000203D4E4D0F045F0C0E0A29192045003AF
:1003E0000203E874010203E9E4D0F045F0B401022D
:1003F00080030203F80203B4E536B401028003026D
:10040000040D8522370536753300B1BD22E536B4BB
:100410000202800302041A0204D1E536B40302800A
:1004200003020427020512E522B40B028003020432
:1004300037053675330022E522B40C02800302042E
:10044000CED1BF85230885240985250A85260B750D
:100450000C0A750D00750E00750F0011686003021F
:10046000046802059A0204CE85230885240985259F
:100470000A85260B790C78277A04116B11686003C2
:100480000204890205EB0204CE8523088524098530
:10049000250A85260B790C782B7A04116B1168607C
:1004A000030204AA0205EB0204CE85230885240971
:1004B00085250A85260B790C782F7A04116B116833
:1004C00060030204CB0205EB0204CE02059A02058A
:1004D00024E522B40C02800302050FD1BF85230856
:1004E00085240985250A85260B790C78277A04113D
:1004F0006B116870030204FB02059AB1BD752300FD
:100500007524007525007526007533000536220216
:100510000524E522B40C028003020524D14CB1BDB0
:100520007539FF220533E533B40802800250030217
:10053000053502059A75080A750900750A00750BDC
:100540000085230C85240D85250E85260F780879D6
:100550000C7A0431368510238511248512258513E4
:1005600026852208750900750A00750B0085230C85
:1005700085240D85250E85260F7808790C7A04319F
:100580002B850C23850D24850E25850F26C0E0784C
:1005900033E6243DF8D0E0A62222053B0538753A23
:1005A0000975355FB1C6E538B4030280030205B9A9
:1005B0007A3C1174753800B1BD7539FF22753A0265
:1005C0007535C8B1C622753401853AF0E53411326B
:1005D00070030205EAC2B3E535311FD2B3E5353108
:1005E0001F0534E53460030205C922753800752300
:1005F00000752400752500752600B1BD742C311FCF
:10060000D2B47A021174C2B47A0111747539FF053B
:100610003B227A041174A290920450030206220233
:100620000648783E7601783F760278407603784136
:100630007604753304753701D14C783E76017533F5
:1006400001753709D14CB1BD7539FF228537F0747A
:100650000AA4C0E0783CD0E0F6753A018533F0E5B5
:100660003A1132700302069C853AF0E53C25F0C051
:10067000E0783DD0E0F6783AE6243DF8E6F535112D
:100680008A74A011F2E53D11F2E53511F211A7745B
:100690000A311F053AE53A600302065C75F009E588
:1006A0003C25F0C0E0783DD0E0F6118A74A011F24C
:1006B000E53D11F2E53311F211A7740A311F2275DD
:1006C000340175F003E534113270030207BF85343D
:1006D000F0740AA4C0E0783CD0E0F67834E6232336
:1006E0002423F8E4F608F608F608F675F009E53C68
:1006F00025F0C0E0783DD0E0F6118A74A011F2E553
:100700003D11F2118A74A111F2D33108F5F085F090
:100710003511A7853533753A018533F0E53A113245
:1007200070030207B6853AF0E53C25F0C0E0783D5D
:10073000D0E0F6118A74A011F2E53D11F2118A742D
:10074000A111F2D33108F5F085F03511A775080A2B
:10075000750900750A00750B00790C7834E62323BF
:100760002423F87A04116B7808790C7A04313678EE
:1007700034E623232423F978107A04116B85350895
:10078000750900750A00750B00790C7834E623238F
:100790002423F87A04116B7808790C7A04312B78C9
:1007A00034E623232423F9780C7A04116B053AE507
:1007B0003A60030207190534E53460030206C222D9
:00000001FF
